:020000040000FA
:0C0000000000000052EF02F067EF02F079
:08001800BCEF02F0106E960E21
:10002000076E980E086E55D8D8B4CA90D8A4CA8066
:10003000FC0FD8A0CA92D8B0CA82800E076E960E66
:10004000086E980E0B6E0C6ACAB025D8CAB223D8B7
:1000500042D80704CB6E07C009F008C00AF0005070
:100060000D6E0E6E003C0E6A4BD80C50102E0AD04E
:10007000BE6E0C0EBD6E0BBEBD8A0BBCBD889394CC
:10008000CA841200BB6E0C0EBA6E0BBEBA8A0BBCD1
:10009000BA889492F5D700D8D8900B32083207323C
:1000A00012000A6A096EFF0E09260A2200D0D8A0A3
:1000B0001200030E086EE60E02D8F5D7086AFE0F8E
:1000C000076EE86A085AD8A012000000070600D0A0
:1000D000F8D70C6A0B6A100EF36E08340B360C3628
:1000E00009500B5C0A500C5805E309500B5E0A508E
:1000F0000C5AD88007360836F32EEFD70750120077
:1001000009500D02F3CF0BF0F4CF0CF00A500D02A2
:10011000F3500C2609500E02F3500C260B5012001F
:100120001B501718226E22BE30D01BBE17D01A509B
:10013000165CD8A0000CD8A4010C1B50175CD8A0EA
:10014000000CD8A4010C1C50185CD8A0000CD8A43A
:10015000010C1D50195CD8A0000C010C16501A5C43
:10016000D8A0000CD8A4010C17501B5CD8A0000C20
:10017000D8A4010C18501C5CD8A0000CD8A4010C09
:1001800019501D5CD8A0000C010C17AE010C000C1E
:10019000800E1B1A1A50165C1F6E11E21F6C16504F
:1001A0001AC016F01A6E17501BC017F01B6E1850AD
:1001B0001CC018F01C6E19501DC019F01D6E1A0ECF
:1001C0001F6074D01A5272E01E6A1750216E1B18FD
:1001D000236E178E1B8E080E1F5E08E31DC01EF0D7
:1001E0001CC01DF01BC01CF01B6AF5D71F2607E0C2
:1001F000D8901B321C321D321E321F2EF9D723AE6F
:1002000033D01D50195E1C50185A1B50175A07E264
:10021000D880000E195618561756800E211A1E6CDB
:1002200004E01906000E185A175A040E1F6E1766BE
:100230000DD018C017F019C018F01EC019F01E6AB2
:10024000080E165E29E31F2EF2D726D017BE08D05F
:10025000D8901E36193618361736162EF7D71CD0FA
:100260001EAE22D01E6A0FD01D5019261C50182217
:100270001B50172206E31732183219321E32164A63
:100280000DD01EAE11D0193E0FD0183E0DD0173E26
:100290000BD0D8801990EFD7166A02D0208216684A
:1002A000196A186A800E176E21AE179E1950120037
:1002B0001750156E1B18236E1A5051E0165252E05B
:1002C000165E7F0E03E2162603E24BD016264CE2A2
:1002D00019C013F018C014F0158E1B8E180E216E65
:1002E000196A186A176A0BD01D50135C1C501458F9
:1002F00011E3146E156A1D50135E0BD004E21B50FF
:10030000155CF2E007E31D50135E1C50145A1B509D
:10031000155AD8801936183617361336143615364E
:10032000212EECD717BE07D016521BE0233216063B
:10033000212A2336E3D707E21D50135E1C50145ABE
:100340001B50155A17E3193E15D0183E13D0173E0F
:1003500011D0173218321932163E0CD005D0208633
:1003600004D02084166A02D020821668196A186A9E
:10037000800E176E23AE179E1950120016C021F082
:10038000175019C017F0196E193621321932206A28
:100390001936213602E32084207E06E12080216A7E
:1003A000196A186A176A0BD0212803E0D88019321D
:1003B00006D0D890193202E1208201D0208620B6E2
:1003C00004D020A20FD020B407D07F0E196EFF0EEC
:1003D000186E176E166E23D0800E196E01D0196A32
:1003E000000EF6D720B0FBD7166A9F0E2160EBD720
:1003F0007E0E2164F4D79E0E215C07E0D89019325E
:10040000183217321632212AF6D720A408D0D88005
:10041000000E165617561856195619AEE0D7165034
:100420001200166E176A186A196A239E0AD0239E54
:1004300019AE07D0D880000E165617561856195602
:10044000238E960E216E195209E0080E212617C040
:1004500016F018C017F019C018F011D018520FE19B
:10046000080E215E175007E1080E215E165002E1CA
:10047000195010D0166A186E16C017F0166A18BEFA
:1004800006D0D8901636173618362106F8D723AE80
:10049000189E215016C019F0166E185017C018F08B
:1004A000176E1200400E206E4F0EAF6E240EAC6E13
:1004B000900EAB6E00010F0EC16E070EB46EC69AA1
:1004C000430E926EE00E936EC00E946E6CD0F2A44A
:1004D00003D0F294817A11009EAA19D0060EAB14B3
:1004E00012E1E2CF5EF0E1CF5DF05F2A10EE81F025
:1004F0005F50E126000EE222AECFE7FF5EC0E2FFD2
:100500005DC0E1FF1100AE50AE50AB98AB8811005A
:100510005F50605C14E0602AEACF08F0E9CF07F092
:1005200000EE81F06050E926000EEA22EF50076EDF
:1005300008C0EAFF07C0E9FFD880120004D0E868CD
:10054000076ED8A0120012005F6A606A9D8A9F8AB7
:10055000F28EF28C12009D9A00EE81F0010EF46E84
:10056000F36AF306000EF45AEE6AF450F310F9E160
:100570005F6A606A9D8A1200F29EE0CF81F3D8CF55
:1005800082F3E8CF83F3F28E0001A192F29E81C341
:10059000E0FF82C3D8FF83C3E8FFF28E10009EA85D
:1005A000FED7AD6E1200939A8A8A0A0E51EC00F0C3
:1005B000939A8A9A94988B9893948A94949A8B9A03
:1005C000006A0F0E0A6EA00E096E020E0EEC00F00D
:1005D000006A0F0E0A6EA00E096E010E0EEC00F0FE
:1005E000929889989296899694908B9094968B96EF
:1005F000406A3F6A3E6A00EE69F0180EEE68E82E27
:10060000FDD7496A426A416A4A6A446A436A4B6A48
:10061000466A456A4C6A486A476A4D6A4E6850683D
:100620004F6A516A646A636A626A616A5050F9DEAD
:1006300019C068F018C067F017C066F016C065F002
:1006400083DF89DFCD6AF294F28A870ED56EB16AB4
:10065000A192A082D08EA292B10EB16E9F90F28C28
:10066000F28E1AEC08F01CEC0AF0562AE86A56B230
:10067000010F57B0010806E15770522A000E5322AD
:100680005422552245DF246EB10E245C06E3FE0E93
:10069000245C01E2266AF5EF05F024AE22D0266A3A
:1006A000800E245C05E124C026F02768286817D056
:1006B000900E245C05E124C026F029682A680FD03A
:1006C000A00E245C05E124C026F02B682C6807D01E
:1006D000B00E245C04E124C026F02D682E68F4EFEF
:1006E00005F0265204E1F5EF05F0F4EF05F0800E79
:1006F000265CD8A441D0272803E124C027F038D0B5
:1007000024C028F07C0E275C09E1929889983E90DD
:100710003F906C686B686A68696827D07D0E275CBB
:1007200009E1929689963E923F9270686F686E6872
:100730006D681BD07E0E275C09E194908B903E94EF
:100740003F9474687368726871680FD07F0E275C7D
:1007500009E194968B963E963F967868776876681E
:10076000756803D02768F5EF05F02768F4EF05F00A
:10077000F5EF05F0F4EF05F0900E265CD8A408D153
:10078000292803E124C029F001D124C02AF02A52EB
:1007900035E17C0E295C09E1929889983E903F9062
:1007A0006C686B686A68696826D07D0E295C09E10F
:1007B000929689963E923F9270686F686E686D68F7
:1007C0001AD07E0E295C09E194908B903E943F9460
:1007D00074687368726871680ED07F0E295C09E1D5
:1007E00094968B963E963F9678687768766875689B
:1007F00002D02968FAD12968F7D1C8D07C0E295CCB
:100800002EE1929889887F0E2A5C22E23E8002EED9
:1008100081F0D8902A34E926000EEA22EECF41F08A
:10082000EFCF42F041505224016E42505320026EED
:10083000000E5420036E000E5520046E04C06CF0B0
:1008400003C06BF002C06AF001C069F03F8006D0BF
:100850003E903F906C686B686A68696895D07D0EC1
:10086000295C2EE1929689867F0E2A5C22E23E82E6
:1008700002EE81F0D8902A34E926000EEA22EECF6B
:1008800043F0EFCF44F043505224016E44505320C4
:10089000026E000E5420036E000E5520046E04C03C
:1008A00070F003C06FF002C06EF001C06DF03F82C7
:1008B00006D03E923F9270686F686E686D6864D033
:1008C0007E0E295C2EE194908B807F0E2A5C22E2C2
:1008D0003E8402EE81F0D8902A34E926000EEA2206
:1008E000EECF45F0EFCF46F045505224016E465012
:1008F0005320026E000E5420036E000E5520046E2D
:1009000004C074F003C073F002C072F001C071F053
:100910003F8406D03E943F9474687368726871682F
:1009200033D07F0E295C2EE194968B867F0E2A5C55
:1009300022E23E8602EE81F0D8902A34E926000EAB
:10094000EA22EECF47F0EFCF48F047505224016E35
:1009500048505320026E000E5420036E000E5520A6
:10096000046E04C078F003C077F002C076F001C0D6
:1009700075F03F8606D03E963F9678687768766831
:10098000756802D0296831D129682ED12ED12CD199
:10099000A00E265C0BE12B2803E124C02BF004D031
:1009A00024C02CF068EC07F020D11ED1B00E265CDC
:1009B000D8A419D12D2803E124C02DF012D124C0D0
:1009C0002EF0400E2D5CD8A492D02EC04DF02E52A9
:1009D00034E08B883E9A3E88006A0F0E0A6EA00EA5
:1009E000096E020E0EEC00F001EE81F0D8902E346C
:1009F000E926000EEA22EECF05F0EFCF06F0055013
:100A00005224016E06505320026E000E5420036ED5
:100A1000000E5520046E04C07CF003C07BF002C0C1
:100A20007AF001C079F04EC000F00F0E0A6EA00EF1
:100A3000096E010E0EEC00F057D03E98006A0F0EC2
:100A40000A6EA00E096E010E0EEC00F07C687B6849
:100A50007A68796851520CE18B98006A0F0E0A6E21
:100A6000A00E096E020E0EEC00F03E9A698A3CD090
:100A7000505011EC02F064C01DF063C01CF062C065
:100A80001BF061C01AF0C8EC00F019C068F018C083
:100A900067F017C066F016C065F068C019F067C04F
:100AA00018F066C017F065C016F0BEEC01F0006EDD
:100AB0000F0E0A6EA00E096E020E0EEC00F0040E70
:100AC0005224016E020E5320026E000E5420036E5B
:100AD000000E5520046E04C080F003C07FF002C0F9
:100AE0007EF001C07DF03E8A2D687ED079D0410E27
:100AF0002D5C0DE1D8902E344E6E4E5206E08B8A5E
:100B00007F0E2E5CD8B44E6801D08B9A69D0420E0D
:100B10002D5C0CE12E5203E1E3EC07F006D05068A7
:100B20004F684E68516A93948A845AD0430E2D5C64
:100B300008E1D8902E34506E7F0E2E5CD8B45068E9
:100B40004FD0440E2D5C2AE12EC051F0505220E0CF
:100B5000515219E0515011EC02F019C01DF018C0AB
:100B60001CF017C01BF016C01AF0505011EC02F028
:100B700058EC01F019C064F018C063F017C062F0BF
:100B800016C061F004D0646A636A626A616A05D063
:100B9000516A646A636A626A616A22D07B0E2D5C64
:100BA0001FE1899889968B908B96006A0F0E0A6ECA
:100BB000A00E096E010E0EEC00F0006A0F0E0A6E18
:100BC000A00E096E020E0EEC00F03E6A406A3F6A0B
:100BD00000EE69F0180EEE68E82EFDD72D6804D0FF
:100BE0002D6803D001D001D039D9060E5C5CD8B095
:100BF0002CD15850525C595053585A5054585B504D
:100C00005558D8A012D15B8E5C5221E13FB007D07D
:100C10003E906C686B686A686968899817D03EA0D6
:100C200015D0807841505224016E42505320026EFC
:100C3000000E5420036E000E5520046E04C06CF0AC
:100C400003C06BF002C06AF001C069F0EDD0010E84
:100C50005C5C21E13FB207D03E9270686F686E68BD
:100C60006D68899617D03EA215D0807643505224E5
:100C7000016E44505320026E000E5420036E000E8D
:100C80005520046E04C070F003C06FF002C06EF017
:100C900001C06DF0C9D0020E5C5C21E13FB407D009
:100CA0003E9474687368726871688B9017D03EA424
:100CB00015D0827045505224016E46505320026E6A
:100CC000000E5420036E000E5520046E04C074F014
:100CD00003C073F002C072F001C071F0A5D0030E22
:100CE0005C5C21E13FB607D03E967868776876680D
:100CF00075688B9617D03EA615D082764750522441
:100D0000016E48505320026E000E5420036E000EF8
:100D10005520046E04C078F003C077F002C076F06E
:100D200001C075F081D0040E5C5C17E13E987C68D0
:100D30007B687A687968006A0F0E0A6EA00E096EE9
:100D4000010E0EEC00F050C000F00F0E0A6EA00E67
:100D5000096E020E0EEC00F067D0050E5C5CD8A4A4
:100D600063D068C019F067C018F066C017F065C09E
:100D700016F064C01DF063C01CF062C01BF061C0BF
:100D80001AF0C8EC00F019C068F018C067F017C07E
:100D900066F016C065F08F0E196EC20E186E750ED5
:100DA000176E780E166E68C01DF067C01CF066C026
:100DB0001BF065C01AF090EC00F0010827E068C055
:100DC00019F067C018F066C017F065C016F0BEECE9
:100DD00001F0006E0F0E0A6EA00E096E020E0EECF0
:100DE00000F0040E5224016E020E5320026E000E1B
:100DF0005420036E000E5520046E04C080F003C022
:100E00007FF002C07EF001C07DF00ED08B983E9A3C
:100E100080697F687E687D68006A0F0E0A6EA00E8A
:100E2000096E020E0EEC00F019D855AE0DD0556AC1
:100E3000546A536A526A3E6A406A3F6A00EE69F039
:100E4000180EEE68E82EFDD706D055AE04D0556AD0
:100E5000546A536A526A807435EF03F05C685B8EA3
:100E6000256A060E255C33E2D8902534E96EEA6ADD
:100E7000EA36E936EA36690EE926000EEA22EFCFB5
:100E800001F0ECCF02F0ECCF03F0ECCF04F05850BF
:100E9000015C595002585A5003585B50045815E2EF
:100EA000D8902534E96EEA6AEA36E936EA36690E00
:100EB000E926000EEA22EFCF58F0ECCF59F0ECCF44
:100EC0005AF0ECCF5BF025C05CF0252ACAE3120093
:100ED0007C0E2B5C1BE12CC049F049520CE002EE69
:100EE00081F0D8904934E926000EEA22EECF41F095
:100EF000EFCF42F00AD0426A416A3F903E906C6860
:100F00006B686A6869688998A9DF59D07D0E2B5C87
:100F10001BE12CC04AF04A520CE002EE81F0D8905E
:100F20004A34E926000EEA22EECF43F0EFCF44F038
:100F30000AD0446A436A3F923E9270686F686E6856
:100F40006D6889968BDF3BD07E0E2B5C1BE12CC03D
:100F50004BF04B520CE002EE81F0D8904B34E92676
:100F6000000EEA22EECF45F0EFCF46F00AD0466AF7
:100F7000456A3F943E9474687368726871688B9098
:100F80006DDF1DD07F0E2B5C1AE12CC04CF04C5253
:100F90000CE002EE81F0D8904C34E926000EEA22F3
:100FA000EECF47F0EFCF48F00AD0486A476A3F9645
:100FB0003E9678687768766875688B964FDF2B6801
:100FC00012002F68120094988B9893948A94949AA4
:100FD0008B9A006A0F0E0A6EA00E096E010E0EECBF
:100FE00000F0006A0F0E0A6EA00E096E020E0EECE3
:100FF00000F0929889989296899694908B90949606
:101000008B96406A3F6A3E6A00EE69F0180EEE6801
:10101000E82EFDD74E685068516A426A416A496AB3
:10102000446A436A4A6A466A456A4B6A486A476A3A
:101030004C6A14D70201826981695C0E846F7A0E52
:10104000836F590E866F850E856F580E886F140E4C
:10105000876F560E8A6FA90E896F550E8C6F430EDF
:101060008B6F530E8E6FE30E8D6F520E906F890E45
:101070008F6F510E926F350E916F4F0E946FE60E7B
:10108000936F4E0E966F9C0E956F4D0E986F580E87
:10109000976F4C0E9A6F190E996F4A0E9C6FDF0E68
:1010A0009B6F490E9E6FAA0E9D6F480EA06F7A0E21
:1010B0009F6F470EA26F4F0EA16F460EA46F290EB1
:1010C000A36F450EA66F080EA56F430EA86FEB0E1B
:1010D000A76F420EAA6FD30EA96F410EAC6FBF0E61
:1010E000AB6F400EAE6FB00EAD6F3F0EB06FA50E82
:1010F000AF6F3E0EB26F9E0EB16F3D0EB46F9C0E81
:10110000B36F3C0EB66F9E0EB56F3B0EB86FA40E5C
:10111000B76F3A0EBA6FAE0EB96F390EBC6FBC0E18
:10112000BB6F380EBE6FCE0EBD6F370EC06FE30EB5
:10113000BF6F360EC26FFD0EC16F360EC46F1A0E32
:10114000C36F350EC66F3B0EC56F340EC86F5F0E92
:10115000C76F330ECA6F870EC96F320ECC6FB20ED7
:10116000CB6F310ECE6FE10ECD6F310ED06F140EFE
:10117000CF6F300ED26F490ED16F2F0ED46F820E0B
:10118000D36F2E0ED66FBE0ED56F2D0ED86FFD0EFF
:10119000D76F2D0EDA6F3F0ED96F2C0EDC6F850ED8
:1011A000DB6F2B0EDE6FCD0EDD6F2B0EE06F180E9A
:1011B000DF6F2A0EE26F670EE16F290EE46FB80E43
:1011C000E36F290EE66F0C0EE56F280EE86F620ED6
:1011D000E76F270EEA6FBC0EE96F270EEC6F180E53
:1011E000EB6F260EEE6F760EED6F250EF06FD80EBC
:1011F000EF6F250EF26F3C0EF16F240EF46FA20E0E
:10120000F36F240EF66F0B0EF56F230EF86F760E4C
:10121000F76F220EFA6FE40EF96F220EFC6F540E78
:10122000FB6F210EFE6FC60EFD6F210E0301006FD6
:101230003B0E0201FF6F200E0301026FB20E016F21
:10124000200E046F2B0E036F1F0E066FA60E056F88
:101250001F0E086F240E076F1E0E0A6FA30E096F74
:101260001E0E0C6F250E0B6F1D0E0E6FA90E0D6F4F
:101270001D0E106F2E0E0F6F1C0E126FB60E116F1B
:101280001C0E146F3F0E136F1B0E166FCB0E156FD7
:101290001B0E186F580E176F1A0E1A6FE80E196F83
:1012A0001A0E1C6F790E1B6F1A0E1E6F0B0E1D6F20
:1012B000190E206FA00E1F6F190E226F360E216FB0
:1012C000180E246FCE0E236F180E266F680E256F32
:1012D000180E286F030E276F170E2A6FA00E296FA6
:1012E000170E2C6F3F0E2B6F160E2E6FDF0E2D6F0D
:1012F000160E306F800E2F6F160E326F240E316F68
:10130000150E346FC80E336F150E366F6E0E356FB7
:10131000150E386F160E376F140E3A6FBF0E396FF9
:10132000140E3C6F690E3B6F140E3E6F150E3D6F31
:10133000130E406FC20E3F6F130E426F710E416F5E
:10134000130E446F210E436F120E466FD20E456F7F
:10135000120E486F840E476F120E4A6F380E496F97
:10136000110E4C6FED0E4B6F110E4E6FA30E4D6FA5
:10137000110E506F5A0E4F6F110E526F120E516FA9
:10138000100E546FCC0E536F100E566F870E556FA4
:10139000100E586F420E576F0F0E5A6F59695C6FDF
:1013A000BD0E5B6F0F0E5E6F7C0E5D6F0F0E606F7C
:1013B0003D0E5F6F0E0E626FFE0E616F0E0E646F5C
:1013C000C00E636F0E0E666F830E656F0E0E686F34
:1013D000470E676F0E0E6A6F0C0E696F0D0E6C6F05
:1013E000D20E6B6F0D0E6E6F990E6D6F0D0E706FCE
:1013F000610E6F6F0D0E726F2A0E716F0C0E746F8F
:10140000F40E736F0C0E766FBE0E756F0C0E786F48
:101410008A0E776F0C0E7A6F560E796F0C0E7C6FFA
:10142000230E7B6F0B0E7E6FF10E7D6F0B0E806FA8
:10143000C00E7F6F000112000101846B340E836FB8
:10144000866B380E856F886B3A0E876F8A6B3C0E01
:10145000896F8C6B3E0E8B6F8E6B400E8D6F906B19
:10146000420E8F6F926B450E916F946B470E936F88
:10147000966B490E956F986B4C0E976F9A6B4F0E4B
:10148000996F9C6B510E9B6F9E6B540E9D6FA06B62
:10149000570E9F6FA26B5A0EA16FA46B5E0EA36FC7
:1014A000A66B610EA56FA86B640EA76FAA6B680E82
:1014B000A96FAC6B6B0EAB6FAE6B6F0EAD6FB06B9D
:1014C000730EAF6FB26B770EB16FB46B7B0EB36FF1
:1014D000B66B800EB56FB86B840EB76FBA6B890EA2
:1014E000B96FBC6B8E0EBB6FBE6B930EBD6FC06BC6
:1014F000980EBF6FC26B9D0EC16FC46BA30EC36FFE
:10150000C66BA80EC56FC86BAE0EC76FCA6BB40EA4
:10151000C96FCC6BBB0ECB6FCE6BC10ECD6FD06BDA
:10152000C80ECF6FD26BCF0ED16FD46BD60ED36FE8
:10153000D66BDE0ED56FD86BE60ED76FDA6BEE0E7C
:10154000D96FDC6BF60EDB6FDE6BDD69010EE06FD1
:10155000080EDF6F010EE26F110EE16F010EE46FF6
:101560001B0EE36F010EE66F250EE56F010EE86FAF
:101570002F0EE76F010EEA6F3A0EE96F010EEC6F66
:10158000450EEB6F010EEE6F500EED6F010EF06F1A
:101590005C0EEF6F010EF26F680EF16F010EF46FCB
:1015A000750EF36F010EF66F820EF56F010EF86F78
:1015B000900EF76F010EFA6F9E0EF96F010EFC6F21
:1015C000AC0EFB6F010EFE6FBB0EFD6F010E020134
:1015D000006FCB0E0101FF6F010E0201026FDB0EE7
:1015E000016F010E046FEC0E036F010E066FFD0E0E
:1015F000056F020E086F0F0E076F020E0A6F210EA5
:10160000096F020E0C6F340E0B6F020E0E6F480E38
:101610000D6F020E106F5D0E0F6F020E126F720EC5
:10162000116F020E146F880E136F020E166F9F0E4D
:10163000156F020E186FB70E176F020E1A6FCF0ECE
:10164000196F020E1C6FE80E1B6F030E1E6F020E49
:101650001D6F030E206F1E0E1F6F030E226F3A0EBA
:10166000216F030E246F570E236F030E266F750E26
:10167000256F030E286F940E276F030E2A6FB40E8A
:10168000296F030E2C6FD50E2B6F030E2E6FF80EE5
:101690002D6F040E306F1C0E2F6F040E326F410E33
:1016A000316F040E346F670E336F040E366F8E0E7B
:1016B000356F040E386FB70E376F040E3A6FE20EB7
:1016C000396F050E3C6F0E0E3B6F050E3E6F3B0EE5
:1016D0003D6F050E406F6A0E3F6F050E426F9B0E09
:1016E000416F050E446FCE0E436F060E466F020E1D
:1016F000456F060E486F380E476F060E4A6F700E24
:10170000496F060E4C6FAA0E4B6F060E4E6FE60E1B
:101710004D6F070E506F240E4F6F070E526F640E01
:10172000516F070E546FA70E536F070E566FEC0ED6
:10173000556F080E586F330E576F080E5A6F7D0E97
:10174000596F080E5C6FC90E5B6F090E5E6F180E45
:101750005D6F090E606F6A0E5F6F090E626FBF0EDC
:10176000616F0A0E646F170E636F0A0E666F720E5A
:10177000656F0A0E686FD00E676F0B0E6A6F310EC1
:10178000696F0B0E6C6F960E6B6F0B0E6E6FFE0E0D
:101790006D6F0C0E706F6A0E6F6F0C0E726FDA0E3B
:1017A000716F0D0E746F4D0E736F0D0E766FC50E4B
:1017B000756F0E0E786F410E776F0E0E7A6FC10E39
:1017C000796F0F0E7C6F460E7B6F0F0E7E6FD00E03
:1017D0007D6F100E806F5E0E7F6F00011200FFD7CD
:020000040030CA
:0300010006160ED2
:020005008580F4
:060008000FC00FE00F40E5
:00000001FF
